:02000000C8280E
:02000E00820767
:10001000023401349D348634823410348134853482
:100020001034843480340F347F3485340F347B347F
:100030007C340F34763486340F34723482340F3487
:1000400074348F340E346334913410345F349A3402
:1000500010345B34473411345534883411345634F9
:100060004934113409346E34B93408348134C93414
:100070000A34713498340B34763483340A34CA34F5
:1000800083340A349A3483340934F13483340834A1
:1000900093349D3407349434B03407347C34AD3415
:1000A00007348534A53408347B34893408348034EB
:1000B00083340734A2349034083447348634073408
:1000C0006034953408348634783407349234873475
:1000D00007349034853407347D34853409345A34F8
:1000E000663409344834663407349E34783408342E
:1000F000BB34603409344C34603408349D3460348B
:1001000009342F3460340734823470340734763441
:10011000703407346634703407346F346A3406340C
:10012000A334703406349834703406348A3470340E
:100130000634723470340434C33499340434B9341A
:10014000993405341C34993403341534203405347F
:100150000F341034013484349D3402341334303479
:1001600003342634503403340F34503402343F34D3
:1001700050340334363420340134683420340334AA
:100180000934203402341A34203402340734203441
:100190008316861705118113FF30860083128B1397
:1001A0008B1506088F000F138F130F088F078F070B
:1001B0000F08072090008F0A0F08072091008F0A70
:1001C0000F080720920010088C0011088E001208FA
:1001D000861BFD28F320051DEE28F12800000515DB
:1001E000E3280511E3288C0BF628FA288D008D0BE7
:1001F000F728F3288E0BFA2808000B106300000084
:040200008B13E8284C
:084000000100020003000400AE
:02400E00F93F78
:1042000054006F006E007900480075006E00740065
:104210002000200056004B003500410048002000DF
:104220004300540043005300530045004E00430038
:1042300020007600200031002E00340020002000F5
:00000001FF
